S31508000000C814002069020008B7080008AF080008ED
S31508000010B308000899040008690D000800000000EC
S31508000020000000000000000000000000B50A0008FB
S31508000030A504000800000000050400089102000855
S31508000040930200089302000893020008930200082E
S31508000050930200089302000893020008930200081E
S31508000060930200089302000893020008930200080E
S3150800007093020008930200089302000893020008FE
S3150800008093020008930200089302000893020008EE
S3150800009093020008930200089302000893020008DE
S315080000A093020008930200089302000893020008CE
S315080000B093020008930200089302000893020008BE
S315080000C093020008930200089302000893020008AE
S315080000D093020008930200089D0C0008930200088A
S315080000E0930200089302000893020008930200088E
S315080000F0930200089302000893020008930200087E
S31508000100930200089302000893020008930200086D
S31508000110930200089302000893020008930200085D
S31508000120930200089302000893020008930200084D
S31508000130930200089302000893020008930200083D
S31508000140930200089302000893020008930200082D
S31508000150930200089302000893020008930200081D
S31508000160930200089302000893020008930200080D
S31508000170930200089302000893020008000000009A
S31508000180930200089302000800F002F800F05CF8F9
S315080001900AA090E8000C82448344AAF10107DA45D4
S315080001A001D100F051F8AFF2090EBAE80F0013F0CA
S315080001B0010F18BFFB1A43F001031847280C00006B
S315080001C0480C00000A444FF0000C10F8013B13F0ED
S315080001D0070408BF10F8014B1D1108BF10F8015B92
S315080001E0641E05D010F8016B641E01F8016BF9D185
S315080001F013F0080F1EBF10F8014BAD1C0C1B09D1DC
S315080002006D1E58BF01F801CBFAD505E014F8016B4D
S3150800021001F8016B6D1EF9D59142D6D370470000DF
S315080002200023002400250026103A28BF78C1FBD8F1
S31508000230520728BF30C148BF0B6070471FB500F092
S3150800024099FD1FBD10B510BD00F065F81146FFF702
S31508000250F5FF00F08DFD00F083F803B4FFF7F2FF19
S3150800026003BC00F083FD0000DFF83400016841F4A8
S3150800027070010160BFF34F8F0A4880470A4800475C
S31508000280FEE7FEE7FEE7FEE7FEE7FEE7FEE7FEE738
S31508000290FEE7FEE705480649044A064B7047000094
S315080002A088ED00E0B90A000889010008C810002096
S315080002B0C8140020C810002072B6704762B670478E
S315080002C072B602B4EFF3118180F31188BFF34F8F32
S315080002D0BFF36F8F084602BC62B6704772B680F3EA
S315080002E01188BFF34F8FBFF36F8F62B6704730BF69
S315080002F0704720BF7047B0FA80F0704790FAA0F0B8
S31508000300B0FA80F0704790FAA0F0704770477047CF
S31508000310704770477047754600F02CF8AE460500E2
S315080003206946534620F00700854618B020B5FFF702
S31508000330B1FFBDE820404FF000064FF000074FF030
S3150800034000084FF0000B21F00701AC46ACE8C009E5
S31508000350ACE8C009ACE8C009ACE8C0098D467047EE
S3150800036010B50446AFF300802046BDE81040FFF7FD
S3150800037074BF0000004870476810002072B64EF639
S315080003802250CEF2000040F2FF01C0F200010170D7
S31508000390002080F3098840F29C00C2F20000016840
S315080003A081F3088800F034FB40F2CA00C2F200006C
S315080003B040F2CB01C2F200010A78027040F2441002
S315080003C0C2F2000040F24811C2F200010A68026057
S315080003D0106880F30988EFF3148040F0020020F0DB
S315080003E0040080F31488BFF36F8FBDE8F04F0FBC8D
S315080003F0BDE8005006BC62B6084726484FF0805153
S315080004000160704772B640F2A002C2F2000211689B
S3150800041081F31188BFF34F8FBFF36F8F62B6EFF387
S3150800042009801EF0100F08BF20ED108A20E9F04F52
S3150800043040F24415C2F2000529680860744600F0C7
S31508000440E7FA40F2CA00C2F2000040F2CB01C2F25B
S3150800045000010A78027040F24811C2F200010A68E7
S315080004602A6044F0040E1068B0E8F04F1EF0100F32
S3150800047008BFB0EC108A80F3098840F20002C0F287
S31508000480000272B682F31188BFF34F8FBFF36F8FE6
S3150800049062B6704704ED00E000BFFEE700BFFEE766
S315080004A000207047704770B50446A56D00F064F8E3
S315080004B0064694F83500022808D08020606500BFFB
S315080004C0002084F8340000BF012070BD2068006851
S315080004D020F01600216808602068406920F0800036
S315080004E021684861206C08B9A06C28B120680068AA
S315080004F020F00800216808602068006820F00100E4
S31508000500216808600FE000F037F8801B05280AD933
S315080005102020606500BF002084F8340000BF032057
S3150800052084F83500D1E72068006800F0010000284B
S31508000530E9D194F85C103F208840A86000BF0020ED
S3150800054084F8340000BF012084F835000020BCE799
S31508000550014691F83500022803D08020486501201D
S315080005607047052081F835000868006820F001000A
S315080005700A6810600020F3E7014800687047000029
S31508000580900000207047704701460022002391F82A
S315080005903D2091F83E3042EA030070472DE9F84FB6
S315080005A00446206805682068C668206847694FF0D1
S315080005B00009CA4605F00F09B9F1000F0AD105F07E
S315080005C0200038B106F0200020B1204600F0B3FA2A
S315080005D0BDE8F88FB9F1000F72D007F0010018B91D
S315080005E006F4907000286BD005F0010030B106F4CF
S315080005F0807018B1206C40F00100206405F00400FA
S3150800060030B107F0010018B1206C40F002002064F8
S3150800061005F0020030B107F0010018B1206C40F077
S315080006200400206405F0080048B106F0200010B95F
S3150800063007F0010018B1206C40F008002064206C17
S3150800064070B305F0200028B106F0200010B120464E
S3150800065000F071FA20684069C0F3801A206C00F037
S31508000660080010B9BAF1000F23D0204600F038FA76
S315080006702068406900F04000402816D1206840698B
S3150800068020F0400021684861A06B50B15648A16B24
S315080006900865A06BFFF75CFF10B1A06B016D88477A
S315080006A00CE02046FFF76FFF08E02046FFF76BFFD8
S315080006B004E02046FFF767FF0020206488E7FFE78D
S315080006C0206B012879D105F01000002875D006F0B6
S315080006D01000002871D000BF002000902068006834
S315080006E0009020684068009000BF00BF20684069FD
S315080006F000F04000402839D1A06B006840681FFA16
S3150800070080F8B8F1000F30D0A08D40452DDDA4F853
S315080007102E80A06BC069B0F5807F1FD02068C068A6
S3150800072020F480702168C8602068406920F00100C4
S31508000730216848612068406920F0400021684861C6
S31508000740202084F83E00002020632068C06820F03E
S3150800075010002168C860A06BFFF7A5FEA08DE28D8A
S31508000760801A81B22046FFF70DFF31E7A08DE18D93
S31508000770401A1FFA80F8E08DE8B1B8F1000F1AD0D8
S315080007802068C06820F490702168C86020684069B5
S3150800079020F0010021684861202084F83E000020EE
S315080007A020632068C06820F010002168C8604146B0
S315080007B02046FFF7E7FE0BE7FFE705F0800030B1BC
S315080007C006F0800018B1204600F037FA00E705F079
S315080007D0400030B106F0400018B1204600F09BF901
S315080007E0F6E600BFF4E60000CD0A000870B5044638
S315080007F00D46164694F83E00202816D105B10EB9C6
S31508000800012070BD00BF94F83C00012801D10220E8
S31508000810F7E7012084F83C0000BF00202063324639
S315080008202946204600F0E6F9EBE70220E9E7000052
S315080008301B49098801F4004189BB1949098801F453
S31508000840804171B1174909780A2903D00021144A51
S31508000850118024E01249098841F40041104A1180A8
S315080008601DE0104909780D2906D10D49098841F47A
S3150800087080410B4A118012E00A490978084A128811
S31508000880C2F30D02084B995405490988491C044AC4
S31508000890118011460988C72901DD0021118070479A
S315080008A004000020060000204C010020704700BF0D
S315080008B0FEE700BFFEE7704770B5002538480078A8
S315080008C0012800D070BD00BF4020FFF7F9FC05469F
S315080008D000BF3448007828B900BF2846FFF7FEFC59
S315080008E000BFEFE72F480078401E2E4908700846DB
S315080008F0007828B100BF2846FFF7F0FC00BFE1E703
S315080009002948007828B100BF2846FFF7E7FC00BF52
S31508000910D8E7264801682648006800F0B7F8044674
S31508000920012C02D0002000F04FF800F0A5F821496C
S3150800093008700846007800EB40001F4951F820006F
S315080009401E490860084600681D49096888420FD193
S31508000950002000F041F80446012C03D0184800682E
S3150800096000F032F800BF2846FFF7B8FC00BFA9E739
S3150800097012480068D0F89400401C10490968C1F86C
S31508000980940010480068401C0E490860FFF735FDC2
S3150800099000BF2846FFF7A2FC00BF00BF92E7000091
S315080009A0A9000020A8000020D6000020940D000809
S315080009B0900D0008CB0000200C0D002048010020F7
S315080009C0440100200401002010B5044600BFFFF7CB
S315080009D065FD00BF10BD000030B504460CB90B48D4
S315080009E00468216A2068884206D3616C206A00EB95
S315080009F081002168884201D8002030BD616C206AD8
S31508000A0000F044F805462846F7E7000044010020B0
S31508000A1070B5FFF745FD054615480068154909688C
S31508000A20884215D012480068D0F89C00281A104948
S31508000A300968C1F898000E480068D0F8A0000C496B
S31508000A400968D1F89810084409490968C1F8A0004E
S31508000A5008480068C0F89C500020FFF7BDFF044610
S31508000A60012C03D002480068FFF7AEFF70BD0000F6
S31508000A70440100204801002010B503490868FFF723
S31508000A803AFCC0B210BD0000CC00002010B50246EA
S31508000A900B46002107E0064C1068A04201D0002052
S31508000AA010BD121D491C0829F5D30120F8E70000DE
S31508000AB04523CDAB704700000348006840F470003A
S31508000AC0014908607047000088ED00E070B50546EA
S31508000AD0AC6B0020E085E0842046FFF754FD70BD2E
S31508000AE00168C96821F490710268D1600168496992
S31508000AF021F0010102685161016B012905D10168E4
S31508000B00C96821F010010268D160202180F83E10E2
S31508000B1000210163704710B504462068C06820F0BC
S31508000B2040002168C860202084F83D002046FFF771
S31508000B30BDFE002010BD70B5044694F83E0022287C
S31508000B4056D1A068B0F5805F0CD1206950B9002550
S31508000B50A66A20684068C0F308003080A06A801C36
S31508000B60A06215E0A56A0026A068B0F5805F03D0EC
S31508000B70A06828B9206918B920684068287004E078
S31508000B802068406800F07F002870A06A401CA062B8
S31508000B90E08D401E80B2E08540BB2068C06820F02A
S31508000BA020002168C8602068C06820F48070216829
S31508000BB0C8602068406920F001002168486120204B
S31508000BC084F83E00206B01280AD12068C06820F00E
S31508000BD010002168C860A18D2046FFF7D3FC02E00B
S31508000BE02046FFF725FE0020206370BD0020FCE7A5
S31508000BF00220FAE710B5034699629A85DA8500203D
S31508000C001864222083F83E0000BF002083F83C00C9
S31508000C1000BF1868C06840F480701C68E0601868F7
S31508000C20406940F001001C6860611868C06840F0BF
S31508000C3020001C68E060002010BD014691F83D00C8
S31508000C40212828D18868B0F5805F0BD1086948B992
S31508000C500A6A1088C0F308000B685860086A801C86
S31508000C60086205E00B6A581C086218780B68586019
S31508000C70C88C401E80B2C88458B90868C06820F07D
S31508000C8080000B68D8600868C06840F040000B68B0
S31508000C90D860002070470220FCE7000070B50024E9
S31508000CA02C4D2D48FFF77AFC00BF03E0641CAC42CC
S31508000CB000D904E02848FFF767FC2028F6D100BFD2
S31508000CC0002403E0641CAC4200D906E00122234953
S31508000CD02148FFF78BFD0028F4D100BF2048FFF715
S31508000CE05DFC002403E0641CAC4200D904E01C4807
S31508000CF0FFF74AFC2028F6D100BF002403E0641C55
S31508000D00AC4200D906E0012214491548FFF76EFDEA
S31508000D100028F4D100BF1348FFF740FC002403E085
S31508000D20641CAC4200D904E00E48FFF72DFC2028CD
S31508000D30F6D100BF002403E0641CAC4200D906E0EB
S31508000D40012206490748FFF751FD0028F4D100BFE4
S31508000D5070BD0000FFFF01001402002006000020FD
S31508000D60580200209C02002000BFFEE700BF704723
S31508000D70002070474FF04070E1EE100A70470000FF
S31508000D80AC0300200600000040000000000100003F
S31508000D90AC040020800000000002000020000000D3
S31508000DA000020000AC0600201E0000000A00000039
S31508000DB0AC0800200A000000640000009001000052
S31508000DC040000000E80300001D0000000A000000C3
S31508000DD03C0A00200C000000800000000002000011
S31508000DE090080000040E0008000000204C010000D6
S31508000DF0C4010008380E00084C0100207C130000CE
S31508000E0020020008814201124C22403B02400C1984
S31508000E1008F202C20C1A482C3C0C0240392908D99F
S31508000E202DB92C3B100158492419080A19042C29F4
S30D08000E302F699001AF000000D4
S7050800018968
